:03000000020013E8
:0C000D00787FE4F6D8FD758132020054C3
:100301000122000123000A103F065B4F666D7D0745
:0B0311007F6F01240001250001260081
:02000B0041A210
:1002A200C0E0C0F0C083C082C0D075D008438CD8F3
:1002B200758AFF052A3131D0D0D082D083D0F0D0D8
:0202C200E03228
:0402C4008E2F8F30BA
:1002C800E4F531F532C3E5329530E531952F500C20
:0C02D80011030532E53270ED053180E9BC
:0102E40022F7
:0700030075A61E75A6E1229F
:10025B00E51DD394175015E51DC39400400EE51E04
:10026B00D3943B5007E51EC394005007E4F51DF5EE
:04027B001EF51C222E
:1001C000E51EC3943A4026E4F51EF51CF521308760
:1001D00005752918800375290D051DE51DC3952991
:1001E000400B208705751D018003E4F51DE51ED336
:0C01F00094025007E4F51EF51CF52122D6
:10017A007F647E0051C4758901C2B9D2A9D28CD2DA
:10018A00AFE4F52AF521515B31C0E4F520F5277576
:10019A002BF9752CA4752D86752EFF711DE52A7015
:1001AA0004110380F8E4F52A11E7711D512D51E578
:0601BA0031FC517F80E7DB
:100131000521E521C39464403FE4F52143200505F1
:100141001CE51C943C4031E4F51C432002051EE5EE
:100151001E943C4023E4F51ED28720870575290DA6
:100161008003752918051DE51DC39529400A2087BF
:0901710004751D0122E4F51D22B4
:0D031D00852BB0852CA0852D90852E80228B
:1000E700E52030E0445320FEE51E75F00A847410C5
:1000F70025F0F8E6F4F52BE51E75F00A842410F8D0
:10010700E6F4F52CE51D75F00A84741025F0F8E681
:10011700F4F52DE51D75F00A842410F8E6F4F52EA4
:0A012700532D7FB4C003752EFF2294
:10009900E51E75F00A84741025F0F8E6F4F52BE5F1
:1000A9001E75F00A842410F8E6F4F52CE51D75F0A8
:1000B9000A84741025F0F8E6F4F52DE51D75F00AAB
:1000C900842410F8E6F4F52E532D7FB4C003752E61
:0E00D900FF852BB0852CA0852D90852E8022D2
:10022D0020A72AE5227026752201D2873087057511
:10023D002918800375290D051DE51DC39529400B52
:0E024D00208705751D018003E4F51D1199221F
:1002E50020B718E5237014752301051EE51EC39478
:0C02F5003C4003E4F51EE4F51C119922C6
:10027F0030A70EE522B401097FE87E0351C4E4F5EF
:10028F002230B70EE523B401097FE87E0351C4E4A1
:03029F00F5232222
:1001FC0020B715E523B401100526D3E526648094B9
:10020C00B24005E4F526F52320A715E522B401102C
:10021C000526D3E526648094B24005E4F526F52244
:01022C0022AF
:1000190002017AE493A3F8E493A34003F68001F282
:1000290008DFF48029E493A3F85407240CC8C333E8
:10003900C4540F4420C8834004F456800146F6DFB7
:10004900E4800B0102040810204080900301E47E43
:10005900019360BCA3FF543F30E509541FFEE493AC
:10006900A360010ECF54C025E060A840B8E493A373
:10007900FAE493A3F8E493A3C8C582C8CAC583CA9E
:10008900F0A3C8C582C8CAC583CADFE9DEE780BE56
:01031C0000E0
:00000001FF
